:100000000C94A4050C94C1050C94C1050C94C10575
:100010000C94C1050C94C1050C94C1050C94C10548
:100020000C94C1050C94C1050C94A72C0C94792D4B
:100030000C9499270C94C1050C94C1050C94C1052E
:100040000C94C1050C94C1050C94C1050C94C10518
:100050000C94C1050C9421280C94C1050C94C10585
:100060000C94C1050C94C1050C94C1050C94C105F8
:100070000C94C1050C94C1050C94C1050C94C105E8
:100080000C94C1050C94C1050C94C1050C94C105D8
:100090000C94C1050C94C1050C94C1050C94C105C8
:1000A0000C94C1050C94C1050C94C1051D091D09D2
:1000B00049094909B109CF09E70AE70ADA09730AC8
:1000C000840A840AA2249824A524ED24F124F1248E
:1000D000ED24F124F124C624F124D024DA24F124DF
:1000E000F124F124F124ED24F124F124ED24F12470
:1000F000B324F124F124EA24EA24EA24EA24EA24B9
:10010000EA24EA24EA24EA24EF24F124A224952410
:10011000F124F124F124F124F124F124F124F12437
:10012000F124F124EF24F124F124ED24F124E82436
:10013000E824E824E824E824E824E824E824E8245F
:10014000EF24E62D0D2E052F0D2E052F592E7C2E7A
:10015000052FD32EE22E2B0014001A0008001500E4
:1001600017001C0018000C00120013002A002900C0
:1001700004001600070009000A000B000D000E0025
:100180000F0033003400E1001D001B0006001900C1
:10019000050011001000360037003800280010510B
:1001A000E000E200E30003512C002C000451500059
:1001B000510052004F002B0014001A0009001300D8
:1001C0000A000D000F0018001C0033002A0029004F
:1001D000040015001600170007000B0011000800AE
:1001E0000C0012003400E1001D001B000600190085
:1001F00005000E00100036003700380028001051AE
:10020000E000E200E30003512C002C0004515000F8
:10021000510052004F002B0034003600370013000D
:100220001C0009000A00060015000F002A00290022
:1002300004001200080018000C0007000B00170053
:10024000110016003800E100330014000D000E000C
:100250001B00050010001A0019001D002800105195
:10026000E000E200E30003512C002C000451500098
:10027000510052004F0035021E021F0220022102CF
:100280002202230224022502260227024C004C00EF
:100290003A003B003C003D003E003F002D022E0294
:1002A0002F023002310201004000410042004300B1
:1002B0004400450032026402010001000100010017
:1002C0000100010001000100010001000100AB007C
:1002D000AA00A900AE0035001E001F00200021006A
:1002E0002200230024002500260027004C004C009B
:1002F0003A003B003C003D003E003F002D002E0038
:100300002F00300031000100400041004200430056
:1003100044004500320064000100010001000100BA
:100320000100010001000100010001000100AB001B
:10033000AA00A900AE0000000000000000000000BC
:1003400000000000000000000000000000000000AD
:10035000000000000000000000000000000000009D
:10036000000000000000000000000000000000008D
:10037000000000000000000000000000000000007D
:100750000000000000000100005C01000100010039
:100760000100010001000100010001004C00010036
:10077000010001001D5C1E5C135C0A5CA75DA85DA6
:10078000A95D01000100010001000100010001005C
:100790000100010001000100010001000100010051
:1007A0000100010001000100010001000100010041
:1007B00001000100010000047F3F1F643214643215
:1007C00014783C1E1E140A052223252628292A2CCB
:1007D0002D2F3032333536383A3B3D3E404243458B
:1007E00047494A4C4E5051535557595A5C5E6062C6
:1007F000646668696B6D6F71737577797B7D7F81D6
:10080000838587898A8C8E90929496989A9C9E9FD5
:10081000A1A3A5A7A8AAACAEAFB1B3B4B6B8B9BBF3
:10082000BCBEBFC1C2C3C5C6C7C9CACBCCCDCED062
:10083000D1D2D2D3D4D5D6D7D7D8D9D9DADADBDB4F
:10084000DBDCDCDCDCDCDDDDDDDDDCDCDCDCDCDBE6
:10085000DBDBDADAD9D9D8D7D7D6D5D4D3D2D2D12F
:10086000D0CECDCCCBCAC9C7C6C5C3C2C1BFBEBC22
:10087000BBB9B8B6B4B3B1AFAEACAAA8A7A5A3A193
:100880009F9E9C9A98969492908E8C8A8987858355
:10089000817F7D7B79777573716F6D6B6968666435
:1008A00062605E5C5A5957555351504E4C4A494705
:1008B000454342403E3D3B3A3836353332302F2DAA
:1008C0002C2A292826252322FFAA7F554000010132
:1008D00001010101010101020202020202020202FF
:1008E00003030303030303030404040404040405CF
:1008F0000505050506060606060707070707080893
:100900000808090909090A0A0A0B0B0B0C0C0C0D43
:100910000D0D0E0E0E0F0F0F1010111111121213DC
:10092000131414151516161717181819191A1A1B57
:100930001B1C1D1D1E1E1F202021222223242425B6
:100940002626272829292A2B2C2D2D2E2F303132EF
:1009500032333435363738393A3B3C3D3E3F4041FF
:1009600042434445464748494A4C4D4E4F505153E7
:1009700054555658595A5B5D5E5F6162646566689E
:10098000696B6C6D6F7072737577787A7B7D7E8022
:1009900082838587888A8C8E8F91939596989A9C6E
:1009A0009EA0A2A3A5A7A9ABADAFB1B3B5B7BABC82
:1009B000BEC0C2C4C6C9CBCDCFD1D4D6D8DBDDDF53
:1009C000E2E4E7E9EBEEF0F3F5F8FAFDFF24035477
:1009D000006800650020006E006F00720069002052
:1009E000004B006500790062006F006100720064D6
:1009F0000000000C03640069003000690062000020
:100A0000000403090409023B00020100A0FA0904E2
:100A10000000010301010009211101000122400031
:100A2000070581030800010904010001030000001B
:100A300009211101000122B60007058203200001EF
:100A4000120100020000000825400C0A44040102C3
:100A5000000105010902A10185020901A1000509A2
:100A60001901290815002501950875018102050164
:100A7000093009311581257F9502750881060938ED
:100A80001581257F950175088106050C0A38021528
:100A900081257F950175088106C0C005010980A1E7
:100AA00001850319012AB700150126B700950175C4
:100AB000108100C0050C0901A101850419012AA0BB
:100AC00002150126A002950175108100C0050109DB
:100AD00006A1018506050719E029E71500250195FE
:100AE00008750181020507190029EF1500250195F8
:100AF000F075018102050819012905950575019117
:100B000002950175039101C005010906A1010507C0
:100B100019E029E715002501950875018102950165
:100B2000750881010507190029FF150026FF0095AA
:100B300006750881000508190129059505750191BB
:100B400002950175039101C011241FBECFEFDAE0B9
:100B5000DEBFCDBF11E0A0E0B1E0E0E9F0E602C009
:100B600005900D92A43CB107D9F723E0A4ECB1E0C5
:100B700001C01D92A331B207E1F70E94FE160C944A
:100B800046300C9400000F9300E124E043E00E9403
:100B900055060F910895FB01883A2DE5920761F003
:100BA000893A2DE5920769F0873A9D4591F4828153
:100BB000882381F080E009C08281882359F081E098
:100BC00004C08281882331F082E00E943B0680E0ED
:100BD000089581E0089581E008950C94CB0508956F
:100BE0000C94EF051F93CF93DF9300D000D01F929A
:100BF000CDB7DEB749835A836B833091C7018981B2
:100C00009A81311114C0662359F0222349F00E94C1
:100C1000240D182F682F89819A810E94CD0C03C062
:100C20000E94F80C182F69817A81812F04C00E94DC
:100C3000240D69817A810F900F900F900F900F9083
:100C4000DF91CF911F910C946914FC01262F4081F4
:100C500051816281738184810C94F20581E0089551
:100C6000CF93DF93EC0160E00E942506BE01DF9187
:100C7000CF910C94F005CF92DF92EF92FF92C12CAE
:100C8000D12C7601C39404C0CC0CDD1CEE1CFF1CDF
:100C90008A95D2F78C2D0E94C611C701B601FF902C
:100CA000EF90DF90CF900C94CF0B8F929F92AF92EA
:100CB000BF92CF92DF92EF92FF920F931F936B013F
:100CC0007C0181E090E0A0E0B0E04C015D0104C057
:100CD000880C991CAA1CBB1C4A95D2F7AC01BD011B
:100CE00004C0440F551F661F771F2A95D2F7482965
:100CF00059296A297B2904C0880F991FAA1FBB1F85
:100D00000A95D2F78A019B010C211D212E213F213A
:100D1000401751076207730739F4BC01CD016C29F4
:100D20007D298E299F290AC080959095A095B09520
:100D3000BC01CD016C217D218E219F211F910F913E
:100D4000FF90EF90DF90CF90BF90AF909F908F90EB
:100D500008950C94AF150C94AB1508950E94770B71
:100D60000E94AD062FEF84E39CE02150804090402C
:100D7000E1F700C000000C9447280F931F93CF9316
:100D8000DF938C0161E00E942506EC01B8010E940E
:100D9000ED05882309F44BC0B801CE010E948221E1
:100DA000882309F444C0B801CE010E94E4258823B9
:100DB000F1F1B801CE010E94A8228823C1F1B80147
:100DC000CE010E944025882391F1B801CE010E94F6
:100DD000C61F882361F1F8018281882309F1CB3590
:100DE0008DE5D807C1F050F4C115FCE5DF0781F0AF
:100DF000CF3DDC45A9F40E94601219C0CC35EDE569
:100E0000DE0761F0CD35DD4559F40E949E1108C022
:100E10000E94AE060CC00E94A71102C00E94AA1137
:100E2000C801DF91CF911F910F910C94EB0580E0E9
:100E3000DF91CF911F910F9108950E947B2780E051
:100E40000E94B7210C943B070E94A6200E943E07F7
:100E50000C94812708950C942A0781E008950C943E
:100E60002D070895CF93C82F0E942B078C2F0E9427
:100E70002F07CF91089580E00C9432070E944026FE
:100E80000C9432070E9440269091C601891721F0E8
:100E90008093C6010C9432070895CF93DF93CDB7AA
:100EA000DEB72B970FB6F894DEBF0FBECDBF4F83D2
:100EB000588769877A878B8761110E94EA109E01A3
:100EC0002F5F3F4F86E0F90111928A95E9F785E09F
:100ED000FE013796D90101900D928A95E1F789813B
:100EE0009A814C815D81452B31F09F3F31F491E037
:100EF0008F3F19F403C091E001C090E090FF09C05A
:100F000049815A816B817C818D819E810E940B1069
:100F100005C0C9010E942E068111F2CF2B960FB693
:100F2000F894DEBF0FBECDBFDF91CF910895FC01D5
:100F3000808191810E94660D0895CF93882309F4E2
:100F4000A9C0C82F8238C1F40E94402681FDA2C0EA
:100F500069E380910201909103010E9436270E946B
:100F60000C112FEF81EE94E0215080409040E1F78A
:100F700000C0000069E319C0833801F50E944026D3
:100F800080FD88C063E580910201909103010E9479
:100F900036270E940C112FEF81EE94E02150804003
:100FA0009040E1F700C0000063E58091020190915C
:100FB00003010E944127CF910C940C118438C1F495
:100FC0000E94402682FD66C067E4809102019091F4
:100FD00003010E9436270E940C112FEF81EE94E04E
:100FE000215080409040E1F700C0000067E4DDCF71
:100FF0008CEF8C0F813AF8F48C2F0E94F72481112A
:1010000049C06C2F80910201909103010E94B62685
:10101000882349F06C2F80910201909103010E9476
:1010200041270E940C116C2F8091020190910301C5
:101030000E943627C0CF80E28C0F883048F4C770FA
:1010400081E001C0880FCA95EAF70E94CD10B3CFA6
:10105000EBE5EC0FE33040F4F0E0E65AFE4F808120
:1010600090E0CF910C947426E8E5EC0FE73150F452
:10107000F0E0EE0FFF1FE45DFE4F80819181CF9184
:101080000C948A26CD3E30F08C2F0E948317CF918E
:101090000C945518CF910895882309F464C08238C0
:1010A00079F40E94402681FF5EC069E380910201CD
:1010B000909103010E9436270E940C1169E310C031
:1010C0008338B1F40E94402680FF4DC063E58091D3
:1010D0000201909103010E9436270E940C1163E5E2
:1010E00080910201909103010E9441270C940C1100
:1010F000843879F40E94402682FF35C067E48091ED
:101100000201909103010E9436270E940C1167E4AE
:10111000E7CF9CEF980F913A10F4682FE1CF90E25F
:10112000980F983050F4877091E001C0990F8A951C
:10113000EAF7892F0E94D310D9CF9BE5980F9330FF
:1011400020F480E090E00C94742698E5980F973195
:1011500020F480E090E00C948A268D3E20F00E94DE
:10116000DE170C94551808951F93CF93DF93182F13
:10117000EB010E949D07209741F08FE99FE00197C6
:10118000F1F700C000002197F6CF812FDF91CF91BA
:101190001F910C944C08893319F060E070E002C094
:1011A00060E570E00C94B408882321F00E94CD1013
:1011B0000C940C110895882321F00E94D3100C94F4
:1011C0000C110895CF92DF92EF92FF920F931F932D
:1011D000CF93DF937C01D62FC72FFC0112810581AD
:1011E00002950F700E94C3108823B9F01123A9F053
:1011F0008C2F807F803421F080E28D0F883068F062
:101200008091CD0282FD09C082E00E946C110E9493
:10121000C31091E0D82ED92601C0D12CCC2EC29477
:101220008FE0C8228C2D90E08C30910508F0CFC162
:10123000FC01EA5AFF4F0C94A12F8C2F807FCF70B6
:10124000882311F0C295C07F112399F0CC2309F4B3
:10125000AAC180E28D0F883010F0D11104C08C2F0C
:101260000E94CD1003C08C2F0E94DD100E940C1133
:101270009AC18D2F0E944C08CC2309F4A8C180E2AA
:101280008D0F883038F1DD2329F18C2F0E94E31077
:1012900024C08C2F807FCF70803211F0C295C07F28
:1012A000DD2319F0D130A1F13DC08091CD0282FF44
:1012B00017C0112349F0CC2329F08C2F0E94CD10A8
:1012C0000E940C1180E070C180E00E944C08CC2389
:1012D00009F47DC18C2F0E94D3100E940C1177C19C
:1012E000112371F0002341F0013031F40E94ED1020
:1012F0008C2B0E94F5106BC10E94ED108C2B1DC031
:10130000002319F0013009F462C10E94021125C0C6
:10131000112321F0063008F05AC10EC0053008F044
:1013200056C11BC0112361F0002331F0F701858104
:1013300080FF39C18F7085838C2F0E94D40847C1EC
:10134000002359F0D93309F03FC1FFEF07EE13E056
:10135000F15000401040E1F735C18C2F0E94DB08AE
:1013600036C18C2F86958695837019F0813061F097
:101370002EC1112321F08D2F9C2F937002C080E08D
:1013800090E00E9474262BC1112321F08D2F9C2FF9
:10139000937002C080E090E00E948A2620C18D2FC9
:1013A000112319F00E94831702C00E94DE170E94C9
:1013B000551815C18C2F837009F047C011110BC14E
:1013C0002D2F229526952770220F220F6D2F6F70DB
:1013D000862F90E0A0E0B0E0022E04C0880F991F95
:1013E000AA1FBB1F0A94D2F7D4FF10C04FE050E0F1
:1013F00060E070E004C0440F551F661F771F2A95F8
:10140000D2F7409550956095709503C040E050E04C
:10141000BA01C695C695C3708A019B01082B192B8A
:101420002A2B3B2BC901B801C23049F058F4C13016
:1014300019F00E94E30BCFC00E94D10BCCC00E94D8
:10144000F50BC9C00E94CF0BC6C0112319F08C2F19
:10145000817001C08695882309F4BDC02D2F229587
:1014600026952770220F220F6D2F6F70862F90E028
:10147000A0E0B0E0022E04C0880F991FAA1FBB1F76
:101480000A94D2F7D4FF10C04FE050E060E070E063
:1014900004C0440F551F661F771F2A95D2F7409549
:1014A00050956095709503C040E050E0BA01C69534
:1014B000C695C3708A019B01082B192B2A2B3B2B45
:1014C000C901B801C23049F058F4C13019F00E9486
:1014D000A80C81C00E94960C7EC00E94BA0C7BC0F2
:1014E0000E94090C78C0CF70112339F08C2F0E9414
:1014F0002F0C8D2F0E94D4086EC08D2F0E94DB0808
:101500008C2F0E94500C67C0D23F21F128F4D03FAD
:1015100041F0D13FC1F043C0D33F19F1D43F79F03E
:101520003EC0112341F0053008F051C08C2F8F715F
:101530000E94750C4CC0063008F049C0F7CF80916E
:10154000CD0282FF18C0112339F08C2F8F710E94B9
:101550002F0C3DC01123C9F38C2F8F710E94500CAA
:1015600036C0112329F08C2F8F710E941A0C2FC0C6
:101570000E94150C2CC0112349F0CF718C2F0E94B2
:101580002F0C63E08C2F0E94511121C081E00E943A
:101590006C110230E0F082E00E946C1118C011233F
:1015A00031F0002391F28D2F0E949D0710C000237F
:1015B00099F2D93349F41FEF27EE33E01150204060
:1015C0003040E1F700C000008D2F0E944C0888EFEA
:1015D0008C0D843020F40E9440260E943207DD20CA
:1015E000C9F00E94BF1080FD15C0F70112820E9451
:1015F000B9100E942F0CC7010E942B0B0E94B9103A
:10160000DF91CF911F910F91FF90EF90DF90CF90DE
:101610000C94500CDF91CF911F910F91FF90EF90A0
:10162000DF90CF9008950F931F93CF93DF93EC013A
:10163000688179818A810E94710D8C010E94CC0C95
:101640000E94BD0BB801CE010E94E208DF91CF914C
:101650001F910F910895CF93DF93EC0198818981B9
:101660002B813C81232B31F08F3F31F481E09F3F70
:1016700019F403C081E001C080E080FD1DC0CE01EF
:101680000E94BD06811110C00E94C3108823A1F0E2
:101690008A81882389F08091CD0282FD0DC082E08D
:1016A000DF91CF910C946C11CE010E94130BCE01EF
:1016B000DF91CF910C943006DF91CF91089580E0B7
:1016C00090E00E94742680E090E00E948A260E94AA
:1016D000EA100E940C110E9486190C9455188091F2
:1016E0000201909103010E944C270C945F0B0E9411
:1016F000DA100C946F0B92959F70963079F010F47D
:10170000925001C09A50923068F4803F69F018F40A
:10171000883E40F409C0843F29F406C0883E20F08A
:10172000813F11F080E0089581E00895FC018081FF
:1017300091810E94660D0E947B0B0895CF93DF93E9
:1017400000D000D01F92CDB7DEB70F900F900F9052
:101750000F900F90DF91CF910895CF93DF9300D03A
:1017600000D000D0CDB7DEB726960FB6F894DEBF16
:101770000FBECDBFDF91CF910895089508950C94C9
:10178000BE0B0C94BF0B0E94C10B6093EA017093D7
:10179000EB018093EC019093ED010C945F0B0C94A2
:1017A000C30B0F931F930091EA011091EB0120915D
:1017B000EC013091ED01602B712B822B932B1F914B
:1017C0000F910C94C30B0F931F930091EA0110919A
:1017D000EB012091EC013091ED0160237123822314
:1017E00093231F910F910C94C30B0F931F930091A0
:1017F000EA011091EB012091EC013091ED0160279D
:101800007127822793271F910F910C94C30B0C947F
:10181000C3050E94070C6093E6017093E701809373
:10182000E8019093E9010C945F0B60E070E0CB015C
:101830000C94090C0F931F9341E050E060E070E0BE
:101840008A019B0104C0000F111F221F331F8A95BC
:10185000D2F7C901B8011F910F910C94090C0F9395
:101860001F9341E050E060E070E004C0440F551F5A
:10187000661F771F8A95D2F78091E6019091E70164
:10188000A091E801B091E9018A019B01082B192B75
:101890002A2B3B2BC901B8011F910F910C94090C05
:1018A0000F931F9341E050E060E070E004C0440FEC
:1018B000551F661F771F8A95D2F740955095609502
:1018C00070958091E6019091E701A091E801B091B7
:1018D000E9018A019B01082319232A233B23C9011B
:1018E000B8011F910F910C94090C0F931F9341E0C5
:1018F00050E060E070E004C0440F551F661F771F82
:101900008A95D2F78091E6019091E701A091E801D4
:10191000B091E9018A019B01082719272A273B2753
:10192000C901B8011F910F910C94090C0F931F93DB
:101930000091E6011091E7012091E8013091E90161
:10194000602B712B822B932B1F910F910C94090C00
:101950000F931F930091E6011091E7012091E80198
:101960003091E90160237123822393231F910F910A
:101970000C94090C0F931F930091E6011091E7015D
:101980002091E8013091E901602771278227932790
:101990001F910F910C94090C08952CE0929F800DDB
:1019A0001124E82FE695E695E695877051E001C091
:1019B000550F8A95EAF785E0E89FF0011124E85376
:1019C000FE4F20E030E070E04081CB01022E02C0EB
:1019D000969587950A94E2F78170819584278523EF
:1019E000842781932F5F3F4F2530310569F7089594
:1019F0002CE0929F800D1124682F66956695669560
:101A0000982F977085E0689FB001112440E050E066
:101A100080E0FB01E40FF51FE853FE4F208130E02A
:101A2000092E02C0369527950A94E2F721703327D4
:101A3000042E01C0220F0A94EAF7822B4F5F5F4FFA
:101A40004530510531F70895BF92CF92DF92EF9262
:101A5000FF920F931F93CF93DF938C01C090E60109
:101A6000D090E701E090E801F090E9018091EA016F
:101A70009091EB01A091EC01B091ED01C82AD92A17
:101A8000EA2AFB2ACFE1D0E0D701C6010C2E04C020
:101A9000B695A795979587950A94D2F780FD04C0CF
:101AA000219790F7B12C07C0BC2EB8018C2F0E9453
:101AB0007C140197A9F38B2DDF91CF911F910F918A
:101AC000FF90EF90DF90CF90BF900895CF93DF937A
:101AD000EC010E94240DBE010E947C14DF91CF9185
:101AE00008951F93CF93DF93EB019091C701992342
:101AF00021F0CB010E94660D13C0882349F0CB0171
:101B00000E94240D182F682FCE010E94CD0C04C016
:101B1000CB010E94F80C182FBE01812F0E947C146B
:101B2000DF91CF911F9108951F93CF93DF93C091C1
:101B3000EE0116E08091EF01C81799F0D0E01C9FEC
:101B4000F0011D9FF00D1124E051FE4F40815181A5
:101B500062817381848195810E94AD0B2196C7704B
:101B6000E9CFDF91CF911F910895409120025091CC
:101B700021026091220270912302809124029091AF
:101B800025020C94AD0BEF92FF920F931F93CF930E
:101B9000DF938091250282958F7009F065C0809156
:101BA0002202882309F460C08091EE01F090EF01D9
:101BB0001091200200912102609123027091240271
:101BC00091E01F3F09F090E0C0910001D091010128
:101BD000292F96E0E92E8F1509F446C0611571058D
:101BE00021F00F3F21F030E003C031E001C0322F7F
:101BF00090E030FD36C0E89EF001E99EF00D112422
:101C0000DF01A051BE4F11963C911197301329C0AE
:101C10003C91311326C012963C911297311121C08C
:101C200013964D915C911497461B570B4C175D070B
:101C3000C0F4809125028F70806180932502EB5063
:101C4000FE4F80818F708061808380E292E00E94ED
:101C50002B0BDF91CF911F910F91FF90EF900C9480
:101C6000940D01968770B7CFDF91CF911F910F919F
:101C7000FF90EF9008959F92AF92BF92CF92DF9224
:101C8000EF92FF920F931F93CF93DF93CDB7DEB701
:101C900061970FB6F894DEBF0FBECDBF8C0185E013
:101CA000F801DE011D9601900D928A95E1F7D801A9
:101CB0001296EC9090912002E09121022091230253
:101CC000309124022115310531F0EF3F31F481E0EC
:101CD0009F3F19F403C081E001C080E0B82FB170CC
:101CE0009B2E80FD47C1D8014C9111965C911197B4
:101CF0001396AD90BC90149780E2C82E82E0D82E47
:101D0000F0902202B501621B730B2091000130910B
:101D10000101FF2009F4D9C08091250262177307E1
:101D200008F095C0282F207F09F052C05E1313C021
:101D3000491311C0FE2CE1100EC08F70806180939A
:101D400025020E94B50DC6010E942B0B8091250231
:101D5000F80185834DC1AB2831F05F3F31F481E05C
:101D60004F3F19F403C081E001C080E080FD03C053
:101D700081E08E2502C080E090E0F82FF170FF2E08
:101D800080FF1CC08091EE012091EF0136E08217A8
:101D900009F40BC190E0389FF001399FF00D112438
:101DA000E051FE4F6181561306C06081461303C0A7
:101DB0006281E61203C001968770E9CFFE2CEE2007
:101DC00009F416C18091250281608093250254C0D8
:101DD0005E1306C0491304C0E11002C0F80199C0A7
:101DE000C8010E94960B882361F1EE2051F12091E9
:101DF0002502822F82958F7090E0029774F0809177
:101E000020029091210298878F831986BB86AA862B
:101E10002C87CE0107960E942B0B86E0F801A0E2EA
:101E2000B2E001900D928A95E1F70E94C30D0E94E5
:101E3000B50D0AC05E1711F1C8010E94960B811101
:101E40002CC0C8010E942B0BFF24F394D1C0282F73
:101E5000207F81F77A2DB98AA88A6E2D89890E9400
:101E60009E0B80E292E00E942B0B86E0D6011D9231
:101E70008A95E9F70E94B50DF12CBAC04913DCCF61
:101E8000E110DACFF8018583C8010E942B0B86E0B0
:101E9000D6011D928A95E9F7ABC0EE2091F2209110
:101EA0002502822F82958F7090E002970CF4B5CFB7
:101EB00080912002909121029A8389831B82BD82A6
:101EC000AC822E83CE010196A6CF6217730708F06D
:101ED00044C0FE2CEE2009F4B4CF5E1330C0491389
:101EE0002EC02091250220FD21C0822F82958F7067
:101EF000482F50E041155105C9F0F80125834F30B6
:101F0000510541F08F5F982F9295907F822F8F70AF
:101F1000892B8583C8010E942B0B86E0F801A0E283
:101F2000B2E001900D928A95E1F73CC086E0F8019D
:101F3000A0E2B2E001900D928A95E1F759C0C80184
:101F40000E94960B811169CF809125028160809358
:101F50002502C8010E942B0B4BC07A2DB98AA88A92
:101F60006E2D89890E949E0B86E0D6011D928A956E
:101F7000E9F718C0EE2009F464CFC8010E94960B5F
:101F8000F82E882309F45DCF86E0F801A0E2B2E0E4
:101F900001900D928A95E1F780E292E00E94970706
:101FA0000E94C30D0E94B50D23C04D875E878D85AD
:101FB0009E850E94660D292F22952F70223028F4CD
:101FC0009F7039F0811105C00BC0243028F49F7038
:101FD00049F4805E883020F0C8010E942B0B9F2CB2
:101FE000F92C06C0D80115969C91907F91F7F8CFF7
:101FF0008F2D61960FB6F894DEBF0FBECDBFDF9177
:10200000CF911F910F91FF90EF90DF90CF90BF90F5
:10201000AF909F9008951F93CF93DF93CDB7DEB716
:102020002C970FB6F894DEBF0FBECDBF4F835887F5
:1020300069877A878B879C87CE0107960E943B0E23
:102040008823D1F09F8188852A853B85232B31F019
:102050008F3F31F481E09F3F19F403C081E001C05C
:1020600080E080FD47C04F81588569857A858B85E2
:102070009C850E94AD0B3EC086E0FE013796DE01D6
:10208000119601900D928A95E1F7FF81E8856A85A6
:102090007B856115710531F0EF3F31F481E0FF3F41
:1020A00019F403C081E001C080E080FD23C02091CD
:1020B000EF0130E0C9010196877099274091EE0148
:1020C00050E084179507F1F1F983EA837D836C83EF
:1020D00096E0929FD001939FB00D1124A051BE4F66
:1020E000FE01319601900D929A95E1F78093EF01F0
:1020F0000E94940D16E08091EE019091EF018917F6
:1021000071F1189FC001112480519E4F0E943B0E17
:10211000882329F1E091EE011E9FF0011124E05186
:10212000FE4F4081518162817381848195810E943B
:10213000AD0B8091EE0190E0019687709927809316
:10214000EE01D9CF0E94770B1092EF011092EE01B1
:10215000E0E2F2E086E0DF011D928A95E9F72C9635
:102160000FB6F894DEBF0FBECDBFDF91CF911F91A8
:10217000089580914602859585958595089580916D
:1021800046028770089590914602977081E009F4A5
:1021900080E0089580916902089590916902892BE9
:1021A00080936902089580959091690289238093B4
:1021B0006902089510926902089590916802892B2E
:1021C0008093680208958095909168028923809396
:1021D0006802089510926802089580914702089558
:1021E00008950C94F0100C94F1109091CD0292FD92
:1021F00008C090914702981721F0809347020C94F1
:10220000F310089580914702882329F01092470225
:1022100080E00C94F3100895CF93DF93E0910201D6
:10222000F0910301809169028083E0910201F091B5
:102230000301908180916802892B808380914702FD
:10224000882381F0E0910201F09103019081892BB4
:10225000808380910201909103010E94A026811148
:102260000E940211C0910201D091030140E250E0AE
:1022700066E272E0CE010E94F12F892B69F080E2C4
:10228000FE01A6E2B2E001900D928A95E1F7CE013F
:10229000DF91CF910C944C26DF91CF9108950C944F
:1022A000F0109091CD0292FD10C098E0899F9001AE
:1022B0001124262B209346020E942F0C8091460267
:1022C0008595859585950C944F110C942F0C109243
:1022D000460280E00C944F112091460280958223A3
:1022E00080934602982F977099F430E0482F082E7B
:1022F000000C550B2417350759F09091CD0292FD33
:1023000007C08595859585950E94500C0C946711A2
:1023100008959091CD0292FB222720F9281769F0A9
:1023200080FB92F99093CD028091CC029091CD02E6
:102330000E94DC1182E00C946C1108958091CD0212
:1023400082FB882780F991E089270C94891181E02C
:102350000C94891180E00C9489116FEF7FEF80E07D
:1023600090E00C94303080E090E00E940C3021E04E
:10237000893E9E4F09F020E0822F089582E090E090
:102380000C94FE2F83E090E00C94FE2F682F83E0E6
:1023900090E00C941230CF9384E090E00E94FE2FE6
:1023A000C82F82E290E00E94FE2F2C2F30E0A9017E
:1023B000582BCA01CF910895CF93C92F682F84E07D
:1023C00090E00E9412306C2F82E290E0CF910C944A
:1023D0001230AB01BC018FE090E00C942430AB01D3
:1023E000BC0183E190E00C94243060E070E0CB010C
:1023F0000C94EF1160E070E0CB010E94E9110C94A5
:10240000F51169EE7EEF80E090E00E94303060E0F0
:1024100082E090E00E94123060E083E090E00E9451
:1024200012301092EA011092EB011092EC0110921E
:10243000ED0160E084E090E00E94123060E082E212
:1024400090E00E94123060E085E090E00E9412303F
:1024500060E086E090E00E9412306FEF87E090E04D
:102460000E94123040E050E0BA0188E090E00E9403
:10247000243060E08DE090E00E94123040E050E0B7
:10248000BA0188E190E00E94243060E087E190E0AA
:102490000E94123040E050E0BA018CE190E00E94CE
:1024A000243060E070E080E290E00E94303040E054
:1024B00050E0BA0188E190E00E9424300C94FA11B7
:1024C0000C940112682F8EE090E00C9412300E9460
:1024D0000628609376027093770280937802909337
:1024E00079026093720270937302809374029093E6
:1024F0007502089585B7806885BF85B7806885BFF8
:10250000089581E008950C94811208950C94851229
:102510000C9485120C9488120C9485120C948C12D5
:102520000C9485120E947A1288E595E10E94362665
:102530000E9490120C948E120E9486120C948512A6
:102540000E9472150E9431070C946D220E94F1279F
:102550000E9457160E94A0120E94A6200E94E51E0B
:102560000C948A125F926F927F928F929F92AF9299
:10257000BF92CF92DF92EF92FF920F931F93CF9370
:10258000DF93CDB7DEB72A970FB6F894DEBF0FBE44
:10259000CDBF0E946C16C82E81110E9467123AE6C8
:1025A000832E32E0932E00E010E0502E802F0E9408
:1025B00096155C01F401619071904F0168267926AF
:1025C00061147104B1F40F5F1F4F0430110569F7F6
:1025D0008FEF89838A831B820E94FA278160782F7C
:1025E0009D838C8349815A816B818D810E944D0727
:1025F0003AC080917A0281FD0E949F15D12CEE2471
:10260000E394F12CC3018E219F21892B29F10E9493
:1026100083128823A9F0DE825F82AE20BF2081E092
:10262000AB2809F480E088870E94FA278160782F20
:102630009A8789874E815F8168858A850E944D07C8
:10264000000F111FF801E659FD4F80819181E826A6
:10265000F926F182E08207C0D394EE0CFF1CFCE067
:10266000DF12D0CFB0CF81E0C11001C080E02A9648
:102670000FB6F894DEBF0FBECDBFDF91CF911F9193
:102680000F91FF90EF90DF90CF90BF90AF909F9011
:102690008F907F906F905F9008950E94B2120E9479
:1026A000181F0E946C220E9473180C944207CF934B
:1026B000DF930E948114EC01811521E5920708F057
:1026C00045C0811530E5930708F094C0883E910518
:1026D00028F5803E910508F0F8C0883A910570F41D
:1026E000853A910508F07CC08130910509F475C0E8
:1026F00008F4E8C0049708F0E8C0E4C08F3B9105F7
:1027000008F0E0C0C85AD0E0CC0FDD1FC35ADE4F3E
:102710000990D881C02DCE019464D8C0811540E2C3
:10272000940758F4811551E0950708F0CEC08D3E0E
:10273000910508F4C7C09065C9C0C11580E4D807E9
:1027400008F4C0C0DF70CE01906AC0C0811525E5D5
:102750009207A8F4811534E5930708F095C0811518
:1027600043E5940708F07BC0811552E5950708F012
:1027700061C0D82FCC27CE01816F906AA7C0C11548
:1027800089E5D807A0F4C11528E5D20708F082C072
:10279000C11536E5D30708F095C08C2F0E9415159A
:1027A0008F7190E0D82FCC27CE0190628FC0C115D9
:1027B0004AE5D40708F474C0CE01905681159042C2
:1027C00008F080C08D2F8F710E941515DD27D06213
:1027D0008F71AE01582BCA0179C081E090E076C0BC
:1027E000C55AD0E0C557DE4F8881C82FD0E0CE0152
:1027F00090646CC074E0969587957A95E1F7282FE0
:1028000023703C2F337081E090E002C0880F991F45
:102810003A95E2F79C68AC01522B9A019C2F9F706D
:102820009695969550E2959FE0011124C9018C2B55
:102830009D2B4CC08370992721E030E002C0220F0D
:10284000331F8A95E2F79C2F9695969580E2989F84
:10285000E0011124C22BD32BCE019C6837C08370BA
:10286000992721E030E002C0220F331F8A95E2F75A
:102870009C2F9695969540E2949FE0011124C22BDF
:10288000D32BCE019A6822C0D82FCC27CE01846FDB
:10289000906A1CC0DC2FCC27CE01806F906A16C0D6
:1028A0008C2F8F700E94151594E0D695C7959A9538
:1028B000E1F7CF70D0E0DC2FCC27D0699E01282B28
:1028C000C90104C080E090E001C0CE01DF91CF914A
:1028D000089520E3829FC0011124FC012CE0729F27
:1028E000E00DF11D1124E60FF11DEE0FFF1FEA5A56
:1028F000FE4F8591949108950E9469140E94571388
:1029000008958238910569F1B0F48133910509F495
:102910006DC048F48932910509F463C08A3291058B
:1029200009F469C008958533910509F455C08933C8
:102930009105B9F00895833E910569F138F4803E20
:102940009105B1F0823E910509F10895863E910509
:10295000A9F1873E9105B9F1843E910509F064C063
:1029600023C02091CC0220FD4FC021FD4DC0089511
:102970008091CC0280FD44C08091CD0280FF44C094
:102980008091CC0284FD42C083EE4DC08091CC0288
:1029900082FF38C0F5CF8091CC0282FD33C0809198
:1029A000CD0280FD31C0ECCF8091CD0281FF32C0DD
:1029B0008091CC0284FD2AC087EE35C08091CC0284
:1029C00083FF26C0F5CF8091CC0283FD21C080918A
:1029D000CD0281FD1FC0ECCF8091CC0285FD1CC0D3
:1029E0001DC08091CC0285FD19C016C08091CC021B
:1029F00086FD16C017C08091CC0286FD13C010C0A2
:102A000089E311C082EE0FC080EE0DC080E00BC0E4
:102A100086EE09C084EE07C089E205C085E303C0E5
:102A20008AE201C081E390E008959091CC0292FF88
:102A30000DC0282F2871283019F4877F846006C0C4
:102A4000282F2471243011F48B7F886093FF0DC0F0
:102A5000282F2871283119F4877E846106C0282F19
:102A60002471243111F48B7E88612091CD0220FFE6
:102A70000DC0382F3871383019F4877F816006C057
:102A8000382F3171313011F48E7F886021FF0DC0F5
:102A9000282F2871283119F4877E816106C0282FDC
:102AA0002171213111F48E7E886194FD877E089515
:102AB00080E008950C94AD110E946C168FE39CE9A0
:102AC0000197F1F700C000000E946C1680E00E94A0
:102AD000961580FF04C00E945A150C94472808954B
:102AE0000C945C150E94B311811102C00E94601207
:102AF0000E94BE1180937A020E94CB119093CD0266
:102B00008093CC020E9470150E94C211682F70E061
:102B100080E090E00E94CF0B6091E6017091E701A8
:102B20008091E8019091E9010C94070CE82FF0E006
:102B3000EE0FFF1FEA52FD4F8081918108950895A5
:102B400080EA8A95F1F7089500C008950C94A015C5
:102B500008950C94A8150C94A9150C94A8150C9420
:102B6000AD15F894E82FE295EF70F0E031A1282F31
:102B70002F7081E090E001C0880F2A95EAF7982F26
:102B80009095932391A392A1892B82A37894089581
:102B90000F931F93CF93DF93CAE9D1E089918F3FC1
:102BA00011F00E94B11581E0CE39D807B9F7CEE80F
:102BB000D1E00AE911E089918F3F11F00E94B1152F
:102BC0000C171D07C1F7DF91CF911F910F91089549
:102BD000BF92CF92DF92EF92FF920F931F93CF930A
:102BE000DF938C01C62FD0E0CE0186569E4F6C013C
:102BF000FC0190819F3F09F450C0B62EF894E92F54
:102C0000E295EF70F0E081A19F7021E030E001C01B
:102C1000220F9A95EAF7822B81A382A1209528237F
:102C200022A378940E94A415EEE8F1E04AE951E06D
:102C300021E030E0E12CF12C61916F3F89F0A62F6B
:102C4000A295AF70B0E090968C9190E06F7002C04A
:102C5000959587956A95E2F780FD02C0C90102C08B
:102C600080E090E0E82AF92A220F331F4E175F0711
:102C700019F7F60180818F3F11F00E94B11561E0D4
:102C8000E114F10409F460E08B2D0E94A615CC0F2D
:102C9000DD1FC00FD11FF982E882DF91CF911F9114
:102CA0000F91FF90EF90DF90CF90BF9008950E941A
:102CB000C81588E0E6EDF2E0DF01982F1D929A95A5
:102CC000E9F7EEECF2E0DF011D928A95E9F784E086
:102CD0000E94B7160C94A906FF920F931F93CF93EF
:102CE000DF93CDB7DEB728970FB6F894DEBF0FBEDF
:102CF000CDBF8E010F5F1F4F88E0F80111928A95BA
:102D0000E9F7F12C6F2DC8010E94E815F394F4E067
:102D1000FF12F8CF48E050E0B8018EEC92E00E943C
:102D2000F12FFF24F394009709F4F12C892B41F043
:102D300088E0F801AEECB2E001900D928A95E1F7DF
:102D40002F2D44E066ED72E08EEC92E00E94B81602
:102D50000E94AB068F2D28960FB6F894DEBF0FBEEB
:102D6000CDBFDF91CF911F910F91FF9008950895EE
:102D7000FF920F931F93CF93DF93F82E092F162FF7
:102D8000D72FC42F222349F081E080937D020E9437
:102D9000FA2790937C0280937B0280917D028823A6
:102DA000D9F080917B0290917C020E9412280597B5
:102DB00098F0EF2DF02FA12FBD2F80E090E04C2F49
:102DC00050E08417950734F4219131912D933D9370
:102DD0000196F7CF10927D02DF91CF911F910F9155
:102DE000FF9008950E94FF290E94A6120C940B2ABE
:102DF0000E940F2A0E944D130C94292A0E949827A2
:102E00000E94E6290E9492120E94F2160E94F81671
:102E10000E949C12FBCF8091840280FF06C06091CB
:102E2000090170E0660F771F26C081FF04C0609122
:102E3000090184E005C082FF07C06091090188E0B4
:102E4000689FB001112417C0909183029923D1F09B
:102E500060910801961788F72091090188E0289F62
:102E600090011124929FA001939F500D112470E0B6
:102E7000CA010E946B2F6038710540F4611571051D
:102E800019F406C068E070E0862F08958FE7089572
:102E900081E008958091840280FF08C0609105015F
:102EA00070E0759567957595679521C081FF06C09F
:102EB0006091050170E07595679519C082FF04C0A7
:102EC0006091050170E010C090918202992399F001
:102ED000609104019617A0F780910501899FC001B8
:102EE000112470E00E946B2F6038710540F4611569
:102EF000710519F406C061E070E0862F08958FE730
:102F0000089581E008958D3E21F40E940B1781956C
:102F100004C08E3E29F40E940B1780938802089506
:102F20008F3E21F40E940B17819504C0803F29F445
:102F30000E940B17809387020895893F19F40E941D
:102F40004A1705C08A3F31F40E944A178195809341
:102F5000890208958B3F21F40E944A17819504C08D
:102F60008C3F29F40E944A1780938A0208959FE0BB
:102F7000980F983078F421E030E0A90102C0440FA6
:102F8000551F9A95E2F7CA0190918602892B80938A
:102F9000860208958D3F21F48091840281600BC0E8
:102FA0008E3F21F480918402826005C08F3F29F416
:102FB0008091840284608093840208958D3E39F468
:102FC0009091880297FF35C01092880259C08E3EBA
:102FD00029F4909188021916BCF32BC090918702B6
:102FE0008F3E29F497FF25C01092870249C0803F89
:102FF00019F41916CCF31DC090918902893F29F468
:103000001916BCF4109289023BC08A3F19F497FF4D
:1030100010C0F8CF8B3F39F490918A0297FF09C016
:1030200010928A022DC08C3F21F490918A021916C9
:10303000BCF39FE0980F983080F421E030E0A901C4
:1030400002C0440F551F9A95E2F7CA0180959091EE
:10305000860289238093860213C08D3F21F48091DC
:1030600084028E7F0BC08E3F21F4809184028D7F7D
:1030700005C08F3F29F4809184028B7F8093840266
:1030800080918702811106C080918802811102C05F
:103090001092830280918902811106C080918A0278
:1030A000811102C01092820208950E94FA27209195
:1030B0008702211104C020918802222321F09093DD
:1030C00081028093800220918902211104C0209105
:1030D0008A02222321F090937F0280937E0285E86A
:1030E00092E00C946626EF92FF920F931F93CF937A
:1030F000DF9300D000D000D0CDB7DEB786E0E5E8A2
:10310000F2E0DE01119601900D928A95E1F7E090D0
:103110008702F09088020091890210918A02109231
:103120008702109288021092890210928A02E1109E
:1031300003C0FF2009F45DC080918002909181025C
:103140000E941228AC0190918302992339F02091BA
:103150000A0130E02417350758F04BC020910B01CD
:103160008AE0289F900111242417350718F041C0E8
:103170009F3F19F09F5F90938302EE2061F00E94C1
:103180000B171E1414F09FEF01C091E0989F902D33
:10319000112490938702FF2061F00E940B171F14E7
:1031A00014F09FEF01C091E0989F902D112490930F
:1031B0008802309187023323E1F020918802222394
:1031C000C1F045EB3403C0011124992319F0909309
:1031D000870203C081E08093870235EB2303C0019F
:1031E0001124992319F09093880203C081E0809301
:1031F0008802011103C0112309F45DC080917E0291
:1032000090917F020E941228AC0190918202992332
:1032100039F02091060130E02417350758F04BC0F3
:10322000209107018AE0289F900111242417350777
:1032300018F041C09F3F19F09F5F909382020023D6
:1032400061F00E944A17101614F09FEF01C091E040
:10325000989F902D112490938902112361F00E9470
:103260004A17111614F09FEF01C091E0989F902D1E
:10327000112490938A02309189023323E1F0209146
:103280008A022223C1F045EB3403C00111249923A3
:1032900019F09093890203C081E08093890235EB95
:1032A0002303C0011124992319F090938A0203C0CB
:1032B00081E080938A028091870281110BC0809106
:1032C0008802811107C080918902811103C0809119
:1032D0008A0281110E945518EB82FC820D831E83A5
:1032E00086E0FE013196A5E8B2E001900D928A9544
:1032F000E1F726960FB6F894DEBF0FBECDBFDF9183
:10330000CF911F910F91FF90EF900895E5E8F2E0C3
:1033100086E0DF011D928A95E9F7109283021092F0
:103320008202109284020895EF92FF920F931F93EE
:10333000CF93DF938B01682F11110AC0442329F02A
:10334000E82FF0E0E353F74F6491762F862F75C096
:10335000212F30E0E82FF0E0442321F0E353F74F32
:10336000E491F0E046E0049FC0011124CFEFD0E0EB
:10337000BE010E94572F4BEA4603C001479F900DA4
:103380001124800F911D800F911D982F990F890F87
:10339000AE01421B530B4E9FD0014F9FB00D5E9F5D
:1033A000B00D11249B2F189FA0011124452F5527E4
:1033B0008E01041B150B0E9FA0010F9F500D1E9F29
:1033C000500D11247E01E81AF108E29E8001E39E6F
:1033D000100DF29E100D1124212F3327C21BD30B89
:1033E000CE9F9001CF9F300DDE9F300D11246230B3
:1033F0007105A9F048F46115710569F06130710536
:10340000C9F48B2F752F0DC06430710581F058F011
:103410006630710579F47E2F8B2F932F0DC0832F8B
:103420007B2F9E2F09C08E2F7B2F952F05C08E2FAF
:10343000732F02C07E2F852F692FDF91CF911F91AF
:103440000F91FF90EF90089541E00E949419089524
:1034500008950E94241A0895CF93DF93762FE901EF
:10346000682F842F0E94291A798368838A83DF91C9
:10347000CF9108958091DE02282F269530E0211506
:10348000310519F48170826005C02532310524F0C0
:10349000817088648093DE02089588E090E00C9447
:1034A0000630CF92DF92EF92FF926B017C010E9477
:1034B0003A1AB701A60188E090E0FF90EF90DF9004
:1034C000CF900C942430EEEDF2E083E08083118203
:1034D0008FEF8283838314826081718182819381E3
:1034E0000C94511A8091DE0280FF02C086950895E7
:1034F00080E008959091E202933018F49F5F9093DA
:10350000E202882351F06091DE027091DF02809127
:10351000E0029091E1020C94511A089581E00C941C
:103520007A1A9091E202992319F091509093E20255
:10353000882351F06091DE027091DF028091E002F9
:103540009091E1020C94511A089581E00C94911A23
:1035500070E00C947D22609110018091DE0280FF6A
:103560000AC080910F0123E0829FC00111248D5178
:103570009D4F0C94A81A8091110190911201891706
:1035800080F7E82FF0E09F01220F331FE20FF31FB7
:10359000ED51FD4F1182108212828F5FF0CF90911A
:1035A000DE0290FF16C09091110120911201921736
:1035B00070F4E92FF0E0DF01AA0FBB1FEA0FFB1F39
:1035C000ED51FD4F8183608342839F5FF0CF0C9468
:1035D000AB1A0895CF93DF9300D01F92CDB7DEB71B
:1035E0009091DE0290FF0AC09E012F5F3F4F0E9424
:1035F0002C1A4B8169818A810E94CF1A0F900F90FB
:103600000F90DF91CF910895CF93DF93EC01EC8180
:10361000F0E0E853F84F4491EEEDF2E062818181F1
:103620000E94EA1A8C818F5F8C83DF91CF9108957D
:10363000CF93DF93EC01EEEDF2E0438162818C8168
:103640000E94EA1A8C818F5F8C83DF91CF9108955D
:103650000F931F93CF93DF9300D01F92CDB7DEB7A8
:103660008C0180918B0281110AC09E012F5F3F4F18
:103670004FEF6FEF0E942C1A8A8180938B02F80122
:103680008481813051F028F0823061F440918B02C6
:103690000AC080918B0240E007C060918B0240E03D
:1036A00080E003C040E080E060E00E94CF1AF801B3
:1036B000848190E0019663E070E00E946B2F848328
:1036C0000F900F900F90DF91CF911F910F91089560
:1036D000AF92BF92CF92DF92EF92FF920F931F9320
:1036E000CF93DF9300D01F92CDB7DEB7182FF62E01
:1036F000042FE22E9091DE0290FF6DC0E92FE69537
:10370000AE2FB0E0A256BE4F8C91809395029E7F63
:10371000923061F49E012F5F3F4F812F0E942C1A3F
:103720004B8169818A810E94CF1A43C0823019F48B
:103730000091E1023EC0863019F41091DF0239C0D9
:103740008930D9F38931A9F5E9518E2F8170D82EAE
:10375000E695F0E0E853F74FA590B490C12CBB2458
:1037600060911301C61618F52C2D30E0A29EC00101
:10377000A39E900DB29E900D112470E00E94572FD1
:10378000812FD11002C0860F01C0861B90911101BC
:10379000290F311DA901440F551F240F351F2D512D
:1037A0003D4F402F6F2D0E942C1AC394D9CF0E94F9
:1037B000AB1A1093DF02F092E0020093E102EE20D8
:1037C00051F06091DE027091DF028091E0029091F1
:1037D000E1020E94511A0F900F900F90DF91CF914C
:1037E0001F910F91FF90EF90DF90CF90BF90AF901F
:1037F0000895EEEDF2E09181282F4381628188E007
:10380000890F0C94681B81E00C94F91BEEEDF2E03B
:103810009181282F4381628188EF890F0C94681B66
:1038200081E00C94061CEEEDF2E0628128E0620F6C
:1038300008F46FEF282F438181810C94681B81E08D
:103840000C94131CEEEDF2E0628128E0621B08F498
:1038500060E0282F438181810C94681B81E00C94E7
:10386000221CEEEDF2E0438128E0420F08F44FEF16
:10387000282F628181810C94681B81E00C94311C9B
:10388000EEEDF2E0438128E0421B08F440E0282FEF
:10389000628181810C94681B81E00C94401C20E0C3
:1038A0000C94681BFF920F931F93CF93DF93EC014F
:1038B000F12C0FEF10E060911301F616F0F48091F7
:1038C00011012F2D30E0280F311DC901880F991FDC
:1038D000280F391F2D513D4F70E0C8010E946B2FFA
:1038E000962F8C814091E1026091E002F99E800D5B
:1038F00011240E942C1AF394DECF0E94AB1A9A81F5
:103900008C8190FF02C08F5F01C081508C83DF915A
:10391000CF911F910F91FF900895AF92BF92CF92D8
:10392000DF92EF92FF920F931F93CF93DF93FC01EF
:10393000828180FF02C00FEF01C001E010E04AE089
:10394000A42E80911301181708F043C08091110133
:10395000C12ED12CE601C80FD11DCE01880F991FB1
:10396000C80FD91FCD51DD4F198218821A8234E059
:10397000E32EF12CB12C80918D028B0D8B302CF02D
:103980006A2D0E94492F892F05C087FF03C090919F
:103990001301890F082E000C990BC816D90691F453
:1039A0008091E1028E9DA0018F9D500D11245595AF
:1039B0004795559547959E016091E0028091DF0201
:1039C0000E942C1AB00EF1E0EF1AF108A1F61F5F69
:1039D000B8CF0E94AB1A80918D02013031F4811171
:1039E00002C080911301815007C090E00196609160
:1039F000130170E00E946B2F80938D02DF91CF91B5
:103A00001F910F91FF90EF90DF90CF90BF90AF90FC
:103A10000895CF938091110190911201891770F44C
:103A2000E82FF0E09F01220F331FE20FF31FED514B
:103A3000FD4F1182108212828F5FF0CFC0E0609143
:103A40001301C617C0F5EC2FF0E070E0CF010E9423
:103A50006B2F20911101820F20918C02022E000CFD
:103A6000330B90E0E217F307CCF020910E01022E09
:103A7000000C330B2E173F078CF09C01220F331FD5
:103A8000820F931F9C012D513D4F4091E1026091A7
:103A9000E0028091DF020E942C1A0BC0FC01EE0FA5
:103AA000FF1F8E0F9F1FFC01ED51FD4F11821082F1
:103AB0001282CF5FC4CF0E94AB1A20910D0180917A
:103AC0008C02820F80938C0290910E01920F909342
:103AD0000E0119165CF4082E000C990B409113018D
:103AE00050E041505109841795071CF0219520930F
:103AF0000D01CF9108958F929F92AF92BF92CF9276
:103B0000DF92EF92FF920F931F93CF93DF938C017D
:103B1000FC014481C42FD0E09E01DE010E94AF2F42
:103B20009B01AC010E94C52F6B017C01E0E2F0E03B
:103B3000EC1BFD0BA5E5B0E09B01AC010E94C52F7D
:103B40004B015C019F01DF010E94A72F9B01AC018B
:103B50000E94D02F9B01AC012C0D3D1D4E1D5F1D01
:103B6000C501B4010E947F2FC22FD22F2A3228F420
:103B7000F3E02F9F900111240DC025E530E02C1BB0
:103B80003109C901880F991F280F391F37FF02C05B
:103B90002F5F3F4F35952795C22FC095F12C85E5B6
:103BA000E82EED1A80911301F816C8F4F1FC02C05A
:103BB0008E2D01C08D2F909111012F2D30E0290FF6
:103BC000311DA901440F551F240F351F2D513D4FA5
:103BD0004C2F6091E0020E942C1AF394E3CF0E94D4
:103BE000AB1AF8018481811102C091E003C08032D8
:103BF00019F49FEF90930C0190910C01890FF8013B
:103C00008483DF91CF911F910F91FF90EF90DF9010
:103C1000CF90BF90AF909F908F9008950F931F9378
:103C2000CF93DF93EC0100E010E080911301282F87
:103C300030E00217130724F5909111019801290F24
:103C4000311DA901440F551F240F351F2D513D4F24
:103C5000869590E04C81081719071CF4442331F035
:103C600002C0411103C04091E10201C040E06091F7
:103C7000E0028091DF020E942C1A0F5F1F4FD5CF08
:103C80000E94AB1A8C8190E00196817099278C83F9
:103C9000DF91CF911F910F910895EEEDF2E08081B9
:103CA0008E7F808360817181828193810E94511A0D
:103CB000109296022FEF80E792E0215080409040D2
:103CC000E1F700C000000C94AB1A6091DE0266952B
:103CD00070E04BE050E084E191E00E94E42F892BFA
:103CE00019F481E0809396020E94FA2790938F0244
:103CF00080938E0208959091DE0290FF35C09170FE
:103D0000811102C0926006C0853210F0986402C032
:103D1000880F982B9093DE02662351F06091DE02AB
:103D20007091DF028091E0029091E1020E94511AAD
:103D30006091DE02669570E04BE050E084E191E036
:103D40000E94E42F892B19F01092960202C00E9463
:103D5000651E81E0809391024091E1026091E00252
:103D60008091DF020C944F1C0895682F9091DE0221
:103D7000969581E0890F853208F081E00C947B1ED6
:103D800081E00C94B51E682F9091DE0296958FEF1E
:103D9000890F09F484E20C947B1E81E00C94C31E0D
:103DA00061E00C947B1EEEEDF2E080818160808307
:103DB00086950C94D01E8091DE0280FD0C944D1EE1
:103DC0000C94D31E60E00C947B1E809194028111B0
:103DD0002EC00E94B311811104C00E9460120E9483
:103DE000631A0E944D1A6093DE027093DF02809383
:103DF000E0029093E1026E7F61F40E94631A0E94D8
:103E00004D1A6093DE027093DF028093E00290937C
:103E1000E1020E943A1A109296028091DE0280FF1F
:103E200003C086950E94E21E81E08093940208956B
:103E30000F931F93CF93DF9380919602882309F409
:103E400085C080919502E091DE02E695E81BE09343
:103E50009002823049F4F0E0EC53F84FE491CE2F19
:103E6000D0E004E01BE149C0863049F4F0E0EF53B4
:103E7000F84FE491CE2FD0E008E11BE13EC089303D
:103E800051F4E695F0E0E254F84FE491CE2FD0E003
:103E900002E51CE132C08F3051F4E695F0E0E554C4
:103EA000F84FE491CE2FD0E00DE81CE126C085311B
:103EB00049F4F0E0E854F84FE491CE2FD0E009E067
:103EC0001DE11BC0883181F0833239F4E6EBF7E065
:103ED000C591D49108E21BE110C0843251F4C4EFC3
:103EE000D1E00EE01EE109C0C8E2D0E00BE71DE121
:103EF00004C0C0EDD7E008E21AE180919102882366
:103F000061F0109291020E94FA2790938F028093A1
:103F10008E0210929302109292020E94FA27E09170
:103F20008E02F0918F028E1B9F0B8F3F9F4770F484
:103F3000EC0FFD1FF0938F02E0938E028EE892E06B
:103F4000F801DF91CF911F910F910994DF91CF91EB
:103F50001F910F910895882311F0FA0101C0FB0110
:103F60000994CF93DF93C82FD62F0E94721A8C1713
:103F700040F00E94721A8D1720F4DF91CF910C94BB
:103F8000C01E8C2FDF91CF910C94D01E1F93CF9326
:103F9000DF93FB0112811111C3C0EC010E94CA1012
:103FA0008272CD3CFCE5DF0709F49AC0A8F5C73C56
:103FB000ECE5DE0709F476C0A8F4C43C9CE5D9071B
:103FC00009F45FC028F4C33CDC4509F457C054C071
:103FD000C53C9CE5D90709F459C0C63CDC4509F449
:103FE0005CC04AC0CA3CFCE5DF0709F46AC050F473
:103FF000C83CECE5DE0709F45AC0C93CDC4509F4CD
:104000005BC03AC0CB3C9CE5D90709F45FC0CC3C0F
:10401000DC4509F460C030C0C23DFCE5DF0709F4AF
:104020006FC088F4CF3C9CE5D90709F460C008F460
:104030005CC0C03DFCE5DF0709F45CC0C13DDC4568
:1040400009F45BC019C0C53D9CE5D90709F460C0FF
:1040500050F4C33DFCE5DF0709F455C0C43DDC4521
:1040600009F454C009C0C63D9CE5D90709F455C000
:10407000CE35DD4509F454C011E052C00E94DB1E6C
:104080004FC04DEC5EE160EC7EE104C040EC5EE1CF
:104090006DEC7EE10E94AB1F43C040E15CE163E058
:1040A0007CE1F8CF43E05CE160E17CE1F3CF4EE2FC
:1040B0005CE16FE17CE1EECF4FE15CE16EE27CE13F
:1040C000E9CF4CE45CE16DE37CE1E4CF4DE35CE1FE
:1040D0006CE47CE1DFCF45EA5AE16EE87AE1DACFC1
:1040E0004EE85AE165EA7AE1D5CF81E017C065E094
:1040F00082E010C068E086E00DC06EE089E00AC092
:1041000064E18FE007C067E185E104C088E106C093
:1041100062E289E10E94B11F03C083E20E94D01EC7
:10412000812FDF91CF911F91089586E090E00C944C
:10413000FE2F682F86E090E00C94123080910103EE
:1041400084708961809301030C9499200E94B311BB
:10415000811104C00E9460120E949E200E9495203E
:1041600080930103282F26952695269530E024304C
:10417000310524F0877088618093010380910103E9
:1041800080FF04C086958695869501C080E00C94DA
:10419000B72120910103822F869586958695482F19
:1041A00050E04330510554F48F5F982F990F990FC9
:1041B000990F822F8770892B8093010380910103CF
:1041C0008160809301030E9499208091010386956C
:1041D000869586950C94B72180910103982F96952A
:1041E00096959695A1F0915E990F990F990F87700A
:1041F000892B80930103887F91E009F490E08091FE
:10420000010390FB80F9809301030E949920809123
:1042100001038695869586950C94B72180910103BC
:1042200080FD13C0816080930103813019F489E01F
:1042300080930103809101030E94992080910103E2
:104240008695869586950C94B721089580910103F3
:1042500080FF08C08E7F809301030E94992080E038
:104260000C94B72108958091010380FD0C942621C0
:104270000C940E2190910103892F86958695869541
:104280008F5F8F719770843038F4880F880F880F94
:10429000892B8093010302C0909301038091010355
:1042A000887F91E009F490E08091010390FB80F910
:1042B000809301030E949920809101038695869541
:1042C00086950C94B721843008F083E09091010327
:1042D0009770282F220F220F220F922B9093010309
:1042E000987F21E009F420E09091010320FB90F9F0
:1042F000909301030C94B7210E94632180910103E4
:104300000C9499209C01FB018281882349F12E3B6A
:10431000FCE53F07C9F040F42C3BECE53E0769F0B3
:104320002D3B3C4561F00895203C9CE5390791F018
:1043300070F0213C3C4589F0089583E001C080E0A5
:104340000E947C2180E008950E94EC20FBCF0E9417
:10435000C920F8CF0E943321F5CF0E943A21F2CF35
:1043600081E00895259A2D9808952D9808958F92AB
:104370009F92AF92BF92CF92DF92EF92FF920F93F4
:104380001F93CF93DF93C82F843050F4811109C05D
:10439000809180008F77809380000E94B52106C0B5
:1043A000C3E080918000806880938000A0918600A7
:1043B000B09187002C2F30E00E94AF2F23E030E037
:1043C00040E050E00E947F2F0027122F232F342F30
:1043D000012F122F232F3327809186009091870081
:1043E0006CE070E00E94572F6017710730F0C80131
:1043F00069E070E00E94572F5EC080918600909126
:104400008700E0908600F0908700E0918600F091B0
:104410008700C6E0D0E0BE010E94572F060F171F8D
:10442000211D311D4801590185E0880C991CAA1CE9
:10443000BB1C8A95D1F7C701BE010E94572F6F019F
:10444000E12CF12CA7019601260F371F411D511DAC
:10445000C501B4010E947F2F69017A01E0918600B5
:10446000F0918700CA01B9010E94392F9B01AC016C
:10447000DF010E94C52F9B01AC01C701B6010E945C
:10448000392FDC01CB012FE0B695A795979587953D
:104490002A95D1F7009186001091870020E030E046
:1044A000081719072A073B0728F4609186007091C6
:1044B0008700CB01BC017093890060938800DF9175
:1044C000CF911F910F91FF90EF90DF90CF90BF9011
:1044D000AF909F908F90089508950E94B22182E836
:1044E0008093800089E1809381008FEF9FEF90930C
:1044F0008700809386000C94A620249A25B12F7EF5
:1045000035B130614FB7F894FC01CB01880F991F8A
:10451000680F791F6E0F7F1FE617F70789F08191EB
:1045200098E035B9000000C087FF25B9880F00006A
:1045300000C000C000C025B900C09A9591F7ECCF2B
:104540004FBF8FE594E00197F1F700C00000089598
:10455000CF93DF93EC01FB018281882309F43CC1F6
:10456000C430FDE5DF0760F4CB3F9CE5D90788F454
:104570009E0122503C452431310508F02EC109C06E
:10458000C236EDE5DE0729F0C63AFDE5DF0709F0A2
:1045900024C10E94CB119093CD028093CC02C131F3
:1045A0008CE5D80709F4C6C008F042C0C930ECE574
:1045B000DE0709F49BC000F5C5308CE5D80709F487
:1045C00085C078F4C330ECE5DE0709F478C008F064
:1045D0007AC0C230DC4509F0F5C08091CC02816020
:1045E000EFC0C7309CE5D90709F478C008F07AC05D
:1045F0008091CC028061E4C0CD30FCE5DF0709F496
:1046000087C058F4CB309CE5D90709F479C008F08D
:104610007BC08091CC0288606FC0CF30FCE5DF07A3
:1046200009F480C008F082C08091CC02877FC8C0A6
:10463000CE3F9CE5D90709F471C000F5C531FCE512
:10464000DF0709F485C068F4C3319CE5D90709F494
:1046500075C008F095C00E94770B8091CC028F77CF
:10466000AFC0CC3FFCE5DF07A9F108F054C0CB3F59
:10467000DC4509F0A7C08091CD0240C0C230EDE515
:10468000DE0709F489C058F4C1158DE5D80709F48F
:104690005AC008F069C08091CD0282602FC0C23636
:1046A000EDE5DE0709F47CC0C63AFDE5DF0709F455
:1046B00081C0C330DD4509F085C080E06EC08091C7
:1046C000CC0282607DC08091CC0216C08091CC0269
:1046D000886076C08091CD0282604FC08091CC020C
:1046E00080626EC08091CC0280646AC00E94770BA9
:1046F0008091CC02806864C0846062C081603DC0EB
:104700008091CC028E7F5CC08091CC028D7F58C09E
:104710008091CC0216C08091CD0218C08091CD024C
:104720008D7F2BC08091CC028F7E4AC08091CC02BD
:104730008F7D46C08091CC028F7B42C08091CC029D
:10474000877F8B7F3DC08091CD028D7F8E7F15C08E
:104750008091CC0282FB222720F991E0922790FBE6
:1047600082F990FB83F92CC08091CD02982F90950F
:1047700091708E7F892B90FB81F98093CD0222C0AE
:104780000E94770B8091CC0287FB222720F991E0D1
:10479000922790FB87F914C081E00E94621212C038
:1047A0008091CC0284FB222720F991E0922790FB94
:1047B00084F906C08091CC02982F909590FB80F9E7
:1047C0008093CC028091CC029091CD020E94DC11AA
:1047D0000E94770B80E001C081E0DF91CF910895C6
:1047E000893289F1F0F4843171F1B0F4873009F045
:1047F00077C081E080930B0184E180930A018AE015
:10480000809309018EE18093080188E0809305017F
:1048100088E28093040164C092EE980F9A30F0F021
:104820005FC0803509F444C028F48F3409F058C0C3
:104830008AE03FC0813529F0823509F051C081E01E
:1048400038C08FEF36C080919902882379F1109299
:104850009902109298021092970242C08D51809353
:104860009902833099F038F4813069F08230D9F4BC
:104870008AE091E00DC0853099F078F0863099F4A7
:1048800084E091E005C08BE091E002C089E091E016
:10489000909398028093970223C088E091E0F8CF2C
:1048A00085E091E0F5CF109299021AC080E008955A
:1048B00086EFE0919702F0919802309789F020817D
:1048C000082E000C990B820F911D8F3F910519F056
:1048D00014F08FEF04C097FF02C0108201C08083E4
:1048E00081E008950F931F9341E050E060E070E095
:1048F0008A019B0104C0000F111F221F331F8A95DC
:10490000D2F7C901B8010E94CF0B1F910F910C94EF
:10491000770B482F50E0FA013597EF33F10508F097
:1049200060C0EE59FF4F0C94A12F0E94601255C039
:1049300080917A02817F8E7F80937A0281E08093DA
:104940009A0208950E94AE0648C080917A02982F7C
:104950009095917090FB80F980937A0291113DC0FF
:10496000897F877F10C080917A0281FB222720F9FE
:1049700091E0922790FB81F980937A02992369F163
:1049800080917A02816080937A0227C080917A02B6
:1049900082FB222720F991E0922790FB82F9ECCF4D
:1049A00080917A0283FB222720F991E0922790FBE5
:1049B00083F9E2CF0E94770B8091CC0287FB2227FC
:1049C00020F991E0922790FB87F98093CC0205C0F3
:1049D000895301C08D510E94722481E0089580E0C6
:1049E000FACF80E0089580E008950C94F324CF93EB
:1049F000C82F80919A02813069F038F08230C1F579
:104A00008C2F0E94F02381E039C00E94CA108232AC
:104A100089F504C00E94CA10823261F48C2F0E9472
:104A2000F524811104C08C2F0E9489241FC081E0CD
:104A300090E01CC08C2F0E94F324811116C0C43159
:104A400089F058F4CB3089F0C031B1F482E0809322
:104A50009A0288E30E94F02308C0C93219F0C833D3
:104A600021F00AC010929A0207C081E0817006C04E
:104A700010929A0280E002C080E0F8CFCF910895B2
:104A8000CF93DF9386319C4541F5EB010E94CA101C
:104A9000982F8A812091020130910301882379F0B7
:104AA0009A7A81E009F480E080939B02911102C020
:104AB00069E201C065E3C9010E9436270AC08091FE
:104AC0009B02811102C069E201C065E3C9010E9435
:104AD00041270E940C1180E001C081E0DF91CF915D
:104AE00008950F931F93CF93DF93C42FD22FFC0110
:104AF00082818823C9F040939E020E94FA279093F6
:104B00009D0280939C0280E28C0F883008F057C091
:104B1000C77081E001C0880FCA95EAF7DF91CF9195
:104B20001F910F910C94D40880919E02481330C0BD
:104B300080919C0290919D020E941228883C9105D0
:104B400038F510E21D0FCD17B9F080E28C0F8830D8
:104B500040F4C77081E001C0880FCA95EAF70E944F
:104B6000DB08183028F581E09D2F977001C0880F71
:104B70009A95EAF70E94D408802F0E94CB0818303B
:104B8000F0F4D77081E001C0880FDA95EAF70AC027
:104B900080E28C0F883098F4C77081E001C0880FE4
:104BA000CA95EAF7DF91CF911F910F910C94DB0822
:104BB000802FDF91CF911F910F910C94CB08DF9143
:104BC000CF911F910F9108950F939C01CB01243F2A
:104BD0004CE5340731F188F4293DFCE53F07D9F075
:104BE0002A3D4CE5340779F1283D3C45A9F506E21C
:104BF00021EE41EE68ED7CE52BC0263FFCE53F074A
:104C0000E1F0A8F0273F3C4539F507E225EE46EEF6
:104C100067EF7CE51DC007E225EE45EE69ED7CE51A
:104C200017C006E221EE40EE64EF7CE511C007E21A
:104C300025EE44EE65EF7CE50BC006E221EE42EE88
:104C400066EF7CE505C008E221E045EE6AED7CE513
:104C50000E94712580E008C0FC018281882319F040
:104C600010929E0201C081E00F9108959093C501BA
:104C70008093C40108959093A4028093A3020895A1
:104C8000E091A302F091A402309721F00190F0810D
:104C9000E02D099480E00895E091A302F091A40230
:104CA000309799F020912B01222359F02091CC02CA
:104CB00027FF07C0DC012C9111962C93119726E059
:104CC0002C930280F381E02D09940895E091A302D2
:104CD000F091A402309739F022E0DC012C9304809B
:104CE000F581E02D099408952091A1023091A2024E
:104CF0002817390771F09093A2028093A102E091E6
:104D0000A302F091A402309721F00680F781E02DF4
:104D10000994089520919F023091A0022817390725
:104D200071F09093A00280939F02E091A302F09112
:104D3000A402309721F00084F185E02D09940895B4
:104D4000FC01329680912B01882331F08091CC02B6
:104D500087FF02C09EE101C096E080E0915028F0FC
:104D600021912223D9F38F5FF9CF0895662351F162
:104D700020912B012223E9F02091CC0227FF19C0BA
:104D8000462F4695469546954E31E0F4677021E0F2
:104D900030E002C0220F331F6A95E2F7FC01E40FF6
:104DA000F11D828190E02823392381E0232B69F4CF
:104DB00009C0FC01329608962191621729F0E81784
:104DC000F907D1F780E0089581E008959C01FC0186
:104DD00032969FEF80E04191461789F09F3F19F48A
:104DE000411101C0982F8F5F8630A9F79F3F39F09E
:104DF000F901E90FF11D97FDFA9562830895089571
:104E00009C012A5F3F4FFC014281461301C0128280
:104E1000019682179307B9F70895262F26952695B0
:104E200026952E3168F4FC01E20FF11D677021E038
:104E300030E001C0220F6A95EAF78281282B228395
:104E40000895262F2695269526952E3170F4FC017F
:104E5000E20FF11D677021E030E001C0220F6A957A
:104E6000EAF72095828128232283089520912B013F
:104E7000222329F02091CC0227FD0C940D270C94BD
:104E8000E62620912B01222329F02091CC0227FD38
:104E90000C9421270C94002720912B01FC013296C1
:104EA000222331F08091CC0287FF02C08EE101C045
:104EB00086E0DF011D928A95E9F7089508950C9424
:104EC0005E2783E08093A5020C945F27811102C0C6
:104ED00081E001C082E08093A5020C945F270C94CE
:104EE000662781E08093A5020C945F270C947127BC
:104EF00008950C9478270C9479270C9478270C94B7
:104F000078270C947827CF930E947F270E946C16F5
:104F10000E947D27C0E08C2F0E949615892B29F4D2
:104F2000CF5FC430C1F780E001C081E0CF91089528
:104F300008951F920F920FB60F9211248F939F9393
:104F4000AF93BF938091A602811113C08091020399
:104F500090910303A0910403B09105034196A11D14
:104F6000B11D8093020390930303A0930403B093B5
:104F70000503BF91AF919F918F910F900FBE0F903E
:104F80001F90189580910A03843031F10E941D070B
:104F90001092A60220E488E190E00FB6F894A8955C
:104FA000809360000FBE2093600083B7817F846090
:104FB00083BF83B7816083BF7894889583B78E7FE2
:104FC00083BF0FB6F894A8958091600088618093A4
:104FD0006000109260000FBE08950E94770B0C9441
:104FE000240782E084BD93E095BD9AEF97BD80933E
:104FF0006E0008952FB7F8948091020390910303F7
:10500000A0910403B09105032FBF08952FB7F89422
:105010006091020370910303809104039091050352
:105020002FBF08959C014FB7F8948091020390918F
:105030000303A0910403B09105034FBF821B930BA0
:10504000089578941F920F920FB60F9211248F93A8
:105050009F93AF93BF938091020390910303A0911C
:105060000403B09105030196A11DB11D80930203B5
:1050700090930303A0930403B0930503BF91AF91F2
:105080009F918F910F900FBE0F901F90189587E7FB
:1050900097E790930108809300089AE088E10FB6A3
:1050A000F894A895809360000FBE90936000FFCFA6
:1050B0008091CA020895089522E02093E9002FEF1D
:1050C0003091E800215035FD06C035ED3A95F1F7F5
:1050D00000002111F5CF2091E80025FF0BC040E032
:1050E00050E066E070E00E949B2A8091E8008E7795
:1050F0008093E8000895CF93DF9320912B01222322
:1051000039F02091CC0227FF03C060E222E002C008
:1051100068E021E02093E9002FEF3091E800215072
:1051200035FD06C035ED3A95F1F700002111F5CFB8
:105130002091E80025FF1DC0EC0180912B01811119
:1051400005C040E050E068E070E003C070E040E07F
:1051500050E0CE010E949B2A8091E8008E778093D8
:10516000E80080E2FE01AAEAB2E001900D928A9581
:10517000E1F7DF91CF9108958093A7027093A90280
:105180006093A80280910A03843001F582E0809345
:10519000E9008FEF9091E800815095FD06C095EDF4
:1051A0009A95F1F700008111F5CF8091E80085FF15
:1051B0000DC040E050E063E070E087EA92E00E94BA
:1051C0009B2A8091E8008E778093E8000895BC01C7
:1051D00084E00C94BC28BC0183E00C94BC28809132
:1051E0000903811109C00E942C2C0E94892C8091F6
:1051F000E20084608093E20008951092090308950C
:105200000C9476276091060381E0611101C080E073
:105210000C94612790910A0381E0943009F080E0BA
:10522000609106030C94662742E061EC81E00E94E5
:10523000A52B42E261EC82E00E94A52B90910A032B
:1052400081E0943009F080E0609106030C946F27B0
:1052500080910C03833009F461C030F4813071F027
:10526000823009F49AC008958A3009F486C08B30E0
:1052700009F46CC0893009F0A8C020C080910B03EC
:10528000813A09F0A2C08091E800877F8093E8000E
:1052900080910F0390911003892B21F460E28AEA38
:1052A00092E003C060E080E090E070E00E94E62AB7
:1052B0008091E8008B778093E800089580910B033C
:1052C000813209F082C080910F0390911003029700
:1052D00008F07BC08091E800877F8093E800809190
:1052E000E80082FD05C080910A038111F8CF6DC0EE
:1052F0002091F3008091F20090E0922B029731F41C
:105300008091F100813011F0863021F48091F1001C
:105310008093CA028091E8008B7753C080910B0381
:10532000813A09F052C080910F0390911003892BAC
:1053300009F04BC08091E800877F8093E80080915E
:10534000E80080FFFCCF80912B0136C080910B03D9
:105350008132D9F580910F0390911003892BA9F523
:105360008091E800877F8093E8000E94DA2B80918B
:105370000D0380932B010C94770B80910B038132EA
:1053800021F58091E800877F8093E8000E94DA2B66
:1053900080910E038093CB02089580910B03813A94
:1053A000A1F48091E800877F8093E8008091E80075
:1053B00080FFFCCF8091CB028093F1008091E800C8
:1053C0008E778093E8000C94DA2B089584B7877F5A
:1053D00084BF0FB6F894A89580916000886180938F
:1053E0006000109260000FBE90E080E80FB6F89465
:1053F00080936100909361000FBE0C9471270E940E
:105400002C2C0E94892CE2EEF0E080818460808365
:1054100078940C941E2F8FE191E00C943B268091A0
:105420000A038530A9F480910A03853079F40E943B
:10543000C227809108038823B1F30E948327882321
:1054400091F30E94852A0E94770BEDCF0C94ED27F3
:10545000089508950C942C2A292F332723303105E1
:10546000C9F060F42130310581F02230310509F0B6
:1054700044C08BE390E025E03AE043C0213231059F
:10548000E1F02232310549F138C082E190E020E4B8
:105490003AE037C099278130910549F028F002970A
:1054A00061F5EDECF9E005C0E1E0FAE002C0E3EF00
:1054B000F9E0849190E09F0124C06115710541F0ED
:1054C00061307105D1F489E090E020E33AE019C041
:1054D00089E090E027E13AE014C06115710541F0E0
:1054E0006130710551F486EB90E022E53AE009C0A5
:1054F00080E490E028E03BE004C080E090E020E021
:1055000030E0FA0131832083089580E189BD82E192
:1055100089BD09B400FEFDCF8091D8008F7D8093B6
:10552000D8008091E00082608093E0008091E000EC
:1055300081FDFCCF0895CF92DF92EF92FF920F93FF
:105540001F93CF93DF93EC018B017A010E94F92B1B
:10555000811133C0E114F10439F0F70180819181A8
:10556000081B190BC80FD91FC12CD12C011511050F
:1055700019F18091E80085FD16C08091E8008E77D2
:105580008093E800E114F10449F0F70180819181F2
:10559000C80ED91ED182C08285E00FC00E94F92BAF
:1055A000882321F30AC089918093F10001501109E9
:1055B000FFEFCF1ADF0ADACF80E0DF91CF911F91A2
:1055C0000F91FF90EF90DF90CF90089520911103FD
:1055D000309112032617370748F06115710539F429
:1055E0002091E8002E772093E80001C0B901FC016A
:1055F00020E06115710579F180910A038823F1F1AA
:105600008530F1F18091E80083FD3CC08091E80095
:1056100082FD2EC08091E80080FFEBCF2091F30047
:105620008091F20090E0922B6115710551F0883065
:10563000910538F421912093F10061507109019690
:10564000F3CF21E0089709F020E08091E8008E7701
:105650008093E800CECF2111CFCF0AC080910A03FA
:10566000882361F0853061F08091E80083FD0AC0F5
:105670008091E80082FFF2CF80E0089582E00895F3
:1056800083E0089581E00895209111033091120381
:105690002617370748F06115710539F42091E800A5
:1056A0002E772093E80001C0B901FC0120E06115CC
:1056B000710591F180910A03882309F440C0853077
:1056C00009F43FC08091E80083FD3DC08091E8006F
:1056D00082FD2FC08091E80080FFE9CF2091F30088
:1056E0008091F20090E0922B6115710559F088309D
:1056F000910540F424912093F10031966150710995
:105700000196F2CF21E0089709F020E08091E800AF
:105710008E778093E800CBCF2111CCCF0AC0809147
:105720000A03882361F0853061F08091E80083FDF1
:105730000AC08091E80082FFF2CF80E0089582E005
:10574000089583E0089581E00895982F973068F5D3
:105750009093E900981739F07091EC002091ED00DA
:105760005091F00003C0242F762F50E021FD02C09D
:105770009F5FECCF3091EB003E7F3093EB00309198
:10578000ED003D7F3093ED003091EB0031603093C0
:10579000EB007093EC002093ED005093F00020910B
:1057A000EE0027FDE5CF80E008958F708093E9003B
:1057B00081E0089580910B0387FF11C08091E8007C
:1057C00082FD05C080910A038111F8CF11C080913C
:1057D000E8008B770BC080910A03882349F0809101
:1057E000E80080FFF8CF8091E8008E778093E80092
:1057F00008952091E4003091E50095E64091EC0099
:10580000842F817040FF23C08091E80080FD1DC07F
:1058100080910A03882399F0853099F08091EB00FC
:1058200085FD11C04091E4005091E5002417350733
:1058300029F3915011F09A01E1CF84E0089582E0BC
:10584000089583E0089581E0089580E008954091EF
:10585000E80042FFDDCF08950E949A2C0E94A22CFE
:10586000E0EEF0E0808181608083E8EDF0E080810F
:105870008F77808319BCA7EDB0E08C918E7F8C93DD
:1058800080818F7E80831092090308950F931F9368
:10589000CF93DF930E949A2C0E94A22CC8EDD0E0F7
:1058A00088818F77888388818068888388818F7DCD
:1058B000888319BC10920A03109206031092080301
:1058C0001092070300EE10E0F80180818B7F808347
:1058D00088818160888342E060E080E00E94A52B9F
:1058E000E1EEF0E080818E7F8083E2EEF0E0808167
:1058F00081608083808188608083F80180818E7FD1
:105900008083888180618883DF91CF911F910F917F
:105910000895E8EDF0E080818F7E8083E7EDF0E090
:1059200080818160808384E082BF81E0809309036D
:105930000C94462CE8EDF0E080818E7F80831092FD
:10594000E20008951092DA001092E10008951F928B
:105950000F920FB60F9211242F933F934F935F93A3
:105960006F937F938F939F93AF93BF93EF93FF9327
:105970008091E10082FF0BC08091E20082FF07C0AE
:105980008091E1008B7F8093E1000E941D2F809128
:10599000DA0080FF1FC08091D80080FF1BC080917B
:1059A000DA008E7F8093DA008091D90080FF0DC0ED
:1059B00080E189BD82E189BD09B400FEFDCF81E0AF
:1059C00080930A030E94EF2805C019BC10920A03B5
:1059D0000E94FD288091E10080FF19C08091E200C3
:1059E00080FF15C08091E2008E7F8093E20080915D
:1059F000E20080618093E2008091D8008062809311
:105A0000D80019BC85E080930A030E940229809186
:105A1000E10084FF30C08091E20084FF2CC080E16F
:105A200089BD82E189BD09B400FEFDCF8091D80017
:105A30008F7D8093D8008091E1008F7E8093E1007C
:105A40008091E2008F7E8093E2008091E20081608D
:105A50008093E20080910603882311F084E007C060
:105A60008091E30087FD02C081E001C083E0809364
:105A70000A030E940A298091E10083FF29C08091D6
:105A8000E20083FF25C08091E100877F8093E100E1
:105A900082E080930A03109206038091E1008E7FDA
:105AA0008093E1008091E2008E7F8093E2008091FC
:105AB000E20080618093E20042E060E080E00E94CA
:105AC000A52B8091F00088608093F0000E9400294F
:105AD000FF91EF91BF91AF919F918F917F916F91C6
:105AE0005F914F913F912F910F900FBE0F901F909C
:105AF00018951F920F920FB60F9211242F933F9378
:105B00004F935F936F937F938F939F93AF93BF93C5
:105B1000CF93DF93EF93FF93C091E900CF70809113
:105B2000EC00D82FD17080FDD0E81092E900809170
:105B3000F000877F8093F00078940E94BD2D109232
:105B4000E9008091F00088608093F000CD2BCF7049
:105B5000C093E900FF91EF91DF91CF91BF91AF9199
:105B60009F918F917F916F915F914F913F912F9175
:105B70000F900FBE0F901F9018951F93CF93DF9338
:105B8000CDB7DEB7AA970FB6F894DEBF0FBECDBF74
:105B9000EBE0F3E08091F100819323E0E331F20741
:105BA000C9F70E9428298091E80083FF2EC18091C7
:105BB0000B0390910C03492F50E04A30510508F037
:105BC00024C1FA01EF55FF4F0C94A12F803821F02A
:105BD000823809F01AC108C0809107039091080328
:105BE000992389F082600FC080910F038F708730F6
:105BF00008F00BC18093E9008091EB0085FB8827BA
:105C000080F91092E9009091E800977F9093E80066
:105C10008093F1001092F100D1C0282F2D7F09F060
:105C2000F4C0882319F0823061F0EFC080910D0339
:105C3000813009F0EAC0933009F080E080930803D6
:105C40002EC080910D0381112AC080910F038F70A7
:105C50002FEF280F263008F0D8C08093E90020915C
:105C6000EB0020FF1CC0933021F48091EB00806298
:105C700014C09091EB0090619093EB0021E030E034
:105C8000A90102C0440F551F8A95E2F74093EA002C
:105C90001092EA008091EB0088608093EB001092F4
:105CA000E9008091E800877F8093E8000E94DA2B6A
:105CB000ACC08111AAC010910D031F778091E30041
:105CC0008078812B8093E3008091E800877F809328
:105CD000E8000E94DA2B8091E80080FFFCCF8091E1
:105CE000E30080688093E300111102C082E001C0EC
:105CF00083E080930A0389C08058823008F085C011
:105D000080910D0390910E038C3D53E0950779F53A
:105D100083E08A838AE289834FB7F894DE01139681
:105D200020E03EE051E2E32FF0E050935700E49191
:105D300020FF03C0E295EF703F5FEF708E2F90E081
:105D4000EA3010F0C79601C0C0968D939D932F5FE7
:105D5000243149F74FBF8091E800877F8093E800A6
:105D60006AE270E0CE0101960E94E62A16C06091B8
:105D70000F0370911003AE014F5F5F4F0E942A2AFC
:105D8000BC01892B09F441C09091E800977F909362
:105D9000E80089819A810E94442B8091E8008B77EA
:105DA0008093E80032C0803881F58091E800877FD9
:105DB0008093E800809106038093F1008091E800D1
:105DC0008E7772CF811121C080910D0390910E03C7
:105DD00099270297D4F48091E800877F8093E800A8
:105DE00080910D03809306030E94DA2B80910603B5
:105DF000811106C08091E30087FD02C081E001C0EF
:105E000084E080930A030E9414298091E80083FFB4
:105E10000AC08091E800877F8093E8008091EB00C2
:105E200080628093EB00AA960FB6F894DEBF0FBE97
:105E3000CDBFDF91CF911F9108950895CF938091A9
:105E40000A038823A1F0C091E900CF709091EC0083
:105E5000892F817090FD80E8C82B1092E900809115
:105E6000E80083FD0E94BD2DCF70C093E900CF9163
:105E70000895DB018F939F930E94C52FBF91AF912F
:105E8000A29F800D911DA39F900DB29F900D112494
:105E9000089587FB082E062687FD819567FD61958D
:105EA0000E94D82F0EF4919507FC81950895AA1BA6
:105EB000BB1B51E107C0AA1FBB1FA617B70710F0F5
:105EC000A61BB70B881F991F5A95A9F78095909527
:105ED000BC01CD01089597FB072E16F4009407D05E
:105EE00077FD09D00E94572F07FC05D03EF490950E
:105EF00081959F4F0895709561957F4F0895A1E218
:105F00001A2EAA1BBB1BFD010DC0AA1FBB1FEE1F33
:105F1000FF1FA217B307E407F50720F0A21BB30B7E
:105F2000E40BF50B661F771F881F991F1A9469F7FA
:105F300060957095809590959B01AC01BD01CF0156
:105F40000895EE0FFF1F0590F491E02D09940E9433
:105F5000AF2F332312F48A1B9B0B0C94C02FA29FEC
:105F6000B001B39FC001A39F700D811D1124911D2D
:105F7000B29F700D811D1124911D08950E94AF2FB5
:105F8000B7FF0895821B930B08950E94AF2FA59F22
:105F9000900DB49F900DA49F800D911D1124089524
:105FA000B7FF0C94C52F0E94C52F821B930B089539
:105FB000991B79E004C0991F961708F0961B881F5B
:105FC0007A95C9F780950895FC014150504030F012
:105FD00001900616D1F73197CF01089588279927A8
:105FE0000895FB01DC0104C08D910190801921F41A
:105FF00041505040C8F7881B990B0895F999FECF7E
:1060000092BD81BDF89A992780B50895A6E1B0E0C8
:1060100044E050E00C943830A8E1B0E042E050E0B9
:106020000C943830262FF999FECF92BD81BDF89A95
:10603000019700B4021639F01FBA20BD0FB6F894CC
:10604000FA9AF99A0FBE08950396272F0E941330EB
:106050000E941230252F0E941330242F0C941330ED
:106060000196272F0E9413300C941230DC01CB01D3
:10607000FC01F999FECF06C0F2BDE1BDF89A319658
:1060800000B40D9241505040B8F70895F894FFCFF6
:10609000C8004802280850011E0A1401010102002C
:1060A0000A000A0A01191A1B1C1D1E1F2021225852
:1060B000287B285C28EB28E7285B2801E200E90020
:1060C000EA00B500B600B700CD008301CC008A011C
:1060D00092019401210223022402250226022702B2
:1060E0002A02B300B4006F007000818283E200E9ED
:1060F00000EA00B500B600B700CD008301CC008AED
:106100000192019401210223022402250226022782
:10611000022A02B300B4006F007000818283F4F59C
:10612000F6F731333236946697C693929190000118
:10613000020202020606060909090909090F0F0FE2
:106140000F0F0F15151518191919191919191919EA
:0461500019232400EB
:00000001FF
